:10000000000000308A006D280F39A8000310A80DE9
:10001000A80D1F08C039280401389F0032302E2057
:100020009F149F1811281E08AB0083161E08831208
:10003000AA00692883178001840AFF3E031D1B283C
:100040006928A501A400FF30A407031CA507031C11
:1000500069280330A300E3302F202328A301F43EB6
:10006000A200A309FE30031C3828A2070318352874
:10007000A2070000A30F3528000022183F282218ED
:1000800041280800A701A6011030A800230DA60DE5
:10009000A70D2408A6022508031C250FA702031894
:1000A00058282408A60725080318250FA7070310BA
:1000B000A20DA30DA80B462822080800A200A31B2E
:1000C000632022086928A209A309A20A0319A30A26
:1000D000080083138312031308008301C0309F00BC
:1000E000713083168F008312850186018701831684
:1000F000811701308500860187010317880083126C
:1001000003139F00803083169F0083128A110A1206
:100110006A29340836028A110A12031D9528330809
:1001200035028A110A12031969298312031333084D
:100130003502A2003408031C013E3602A3008A01E6
:100140005F20A0002308A100033021028A110A12B7
:10015000031CB4288A110A12031DB628E9302002B4
:100160008A110A120318B6280301031D01308312F5
:100170000313B000B6088A110A12031DC5281030F7
:1001800035028A110A12031CC7280301031D01301E
:1001900083120313B0048A110A120319D2288A1198
:1001A0000A12122933083502A2003408031C013E4A
:1001B0003602A3008A015F20A0002308A100A10845
:1001C0008A110A12031DEA28103020028A110A122D
:1001D000031C192983120313340CAB00330CAA003F
:1001E000AB0CAA0CAB0CAA0CAB0CAA0C0F30AB05D9
:1001F0002A083302B3002B08031C013E3402B4006A
:10020000360CAB00350CAA00AB0CAA0CAB0CAA0C3C
:10021000AB0CAA0C0F30AB052A08B3072B08031848
:10022000013EB4073608B4003508B3008A110A123B
:1002300065293408AB003308AA003408AD00330840
:10024000AC00AF011030AE000310AF0CAE0C0310C9
:10025000AF0CAE0C2D08A3002C08A2002F08A5009F
:100260002E08A4008A014220AC002308AD002C080F
:100270002A02B3002D08031C013E2B02B4003408EF
:10028000AB003308AA003608AD003508AC00AF015A
:100290001030AE000310AF0CAE0C0310AF0CAE0C60
:1002A0002D08A3002C08A2002F08A5002E08A400EA
:1002B0008A014220AC002308AD002A082C07B300B5
:1002C0002B080318013E2D07B4003408B60033088C
:1002D000B500080064308A0121202030840060309D
:1002E0008A011B20A030840050308A011B2010306E
:1002F000840060308A011A209030840060308A01C6
:100300001A2083168711831287118316071183120F
:100310000711831687108312871083160710831224
:100320000710831605138312051383168513831292
:100330008513831685128312851283160512831284
:1003400005128316851183128511831605118312F8
:100350000511831685108312851083168613831268
:1003600086138316071283120712831687128312CD
:10037000871283160713831207138316071083123D
:100380000710831606108312061083168610831238
:1003900086108316061183120611831686118312A6
:1003A0008611831606128312061283168612831292
:1003B0008612831606138312061300308A01042066
:1003C000B1002B08B2003208B6003108B5008A012E
:1003D00089203608B2003508B100B2088A110A1225
:1003E000031DFE29323031028A110A120318FE2938
:1003F0008501860187018A110A12242DB2088A110B
:100400000A12031D092A323031028A110A12031C12
:100410001D2A83120313B2088A110A12031D1D2A12
:10042000643031028A110A1203181D2A85018601DF
:10043000083087008A110A12242DB2088A110A1284
:10044000031D282A643031028A110A12031C3C2A37
:1004500083120313B2088A110A12031D3C2A963034
:1004600031028A110A1203183C2A850186010C30D8
:1004700087008A110A12242DB2088A110A12031D5C
:10048000472A963031028A110A12031C5B2A831212
:100490000313B2088A110A12031D5B2AC830310205
:1004A0008A110A1203185B2A850186010E30870023
:1004B0008A110A12242DB2088A110A12031D662A13
:1004C000C83031028A110A12031C7A2A83120313DC
:1004D000B2088A110A12031D7A2AFA3031028A11EF
:1004E0000A1203187A2A850186010F3087008A11C3
:1004F0000A12242DB2088A110A12031D852AFA3025
:1005000031028A110A12031CA12A0130831203133B
:1005100032028A110A12031C972A8A110A12031D39
:10052000A12A2C3031028A110A120318A12A403064
:1005300083120313850086010F3087008A110A1287
:10054000242D013032028A110A12031CCD2A8A118D
:100550000A12031DB12A2C3031028A110A12031C1F
:10056000CD2A01308312031332028A110A12031CAE
:10057000C32A8A110A12031DCD2A5E3031028A1164
:100580000A120318CD2AC030831203138500860196
:100590000F3087008A110A12242D013032028A118D
:1005A0000A12031CF92A8A110A12031DDD2A5E3081
:1005B00031028A110A12031CF92A01308312031333
:1005C00032028A110A12031CEF2A8A110A12031D31
:1005D000F92A903031028A110A120318F92AE03000
:1005E00083120313850086010F3087008A110A12D7
:1005F000242D013032028A110A12031C252B8A1184
:100600000A12031D092B903031028A110A12031CB1
:10061000252B01308312031332028A110A12031CA4
:100620001B2B8A110A12031D252BC23031028A119D
:100630000A120318252BF03083120313850086015C
:100640000F3087008A110A12242D013032028A11DC
:100650000A12031C512B8A110A12031D352BC230BA
:1006600031028A110A12031C512B01308312031329
:1006700032028A110A12031C472B8A110A12031D27
:10068000512BF43031028A110A120318512BF83021
:1006900083120313850086010F3087008A110A1226
:1006A000242D013032028A110A12031C7D2B8A117B
:1006B0000A12031D612BF43031028A110A12031C45
:1006C0007D2B02308312031332028A110A12031C9B
:1006D000732B8A110A12031D7D2B263031028A11D9
:1006E0000A1203187D2BFC30831203138500860148
:1006F0000F3087008A110A12242D023032028A112B
:100700000A12031CA92B8A110A12031D8D2B2630F5
:1007100031028A110A12031CA92B0230831203131F
:1007200032028A110A12031C9F2B8A110A12031D1E
:10073000A92B583031028A110A120318A92BFE3056
:1007400083120313850086010F3087008A110A1275
:10075000242D023032028A110A12031CD62B8A1170
:100760000A12031DB92B583031028A110A12031CD8
:10077000D62B02308312031332028A110A12031C91
:10078000CB2B8A110A12031DD62B8A3031028A1113
:100790000A120318D62BFE30831203138500803013
:1007A00086000F3087008A110A12242D023032028F
:1007B0008A110A12031C032C8A110A12031DE62B4C
:1007C0008A3031028A110A12031C032C0230831270
:1007D000031332028A110A12031CF82B8A110A121F
:1007E000031D032CBC3031028A110A120318032C9A
:1007F000FE30831203138500803086001F3087008F
:100800008A110A12242D023032028A110A12031CA4
:10081000302C8A110A12031D132CBC3031028A11AC
:100820000A12031C302C02308312031332028A1185
:100830000A12031C252C8A110A12031D302CEE30DB
:1008400031028A110A120318302CFE30831203136E
:100850008500803086003F3087008A110A12242DDF
:10086000023032028A110A12031C5D2C8A110A120C
:10087000031D402CEE3031028A110A12031C5D2C3C
:1008800003308312031332028A110A12031C522C02
:100890008A110A12031D5D2C203031028A110A12BE
:1008A00003185D2CFE308312031385008030860010
:1008B0007F3087008A110A12242D033032028A11F8
:1008C0000A12031C8A2C8A110A12031D6D2C203077
:1008D00031028A110A12031C8A2C0330831203137B
:1008E00032028A110A12031C7F2C8A110A12031D7C
:1008F0008A2C523031028A110A1203188A2CFE30D7
:1009000083120313850080308600FF3087008A1130
:100910000A12242D033032028A110A12031CB72C4A
:100920008A110A12031D9A2C523031028A110A12BE
:10093000031CB72C03308312031332028A110A12EC
:10094000031CAC2C8A110A12031DB72C843031020F
:100950008A110A120318B72CFE3083120313850084
:1009600081308600FF3087008A110A12242D03305F
:1009700032028A110A12031CE42C8A110A12031D86
:10098000C72C843031028A110A12031CE42C033074
:100990008312031332028A110A12031CD92C8A1102
:1009A0000A12031DE42CB63031028A110A12031810
:1009B000E42CFE3083120313850083308600FF3061
:1009C00087008A110A12242D033032028A110A127A
:1009D000031C112D8A110A12031DF42CB6303102AA
:1009E0008A110A12031C112D0330831203133202E1
:1009F0008A110A12031C062D8A110A12031D112DD9
:100A0000E83031028A110A120318112DFE308312C8
:100A10000313850087308600FF3087008A110A1291
:100A2000242DB2088A110A12031D1C2D65303102D3
:100A30008A110A12031C242DFE3083120313850031
:100A40008F308600FF3087008A01DD298A01262D3C
:02400E00A42CE0
:02401000FF3F70
:00000001FF
